:020000040000FA
:1000000000040020990900002D0600007909000075
:1000100037060000410600004B060000000000000B
:10002000000000000000000000000000BD0900000A
:1000300055060000000000005F0600006906000091
:10004000730600007D060000870600009106000090
:100050009B060000A5060000AF060000B9060000E0
:10006000C3060000CD060000D7060000E106000030
:10007000EB060000F5060000FF060000090700007F
:10008000130700001D0700002707000031070000CC
:100090003B070000450700004F070000590700001C
:1000A000630700006D07000077070000810700006C
:1000B0008B070000950700009F070000A9070000BC
:1000C000B3070000BD070000C7070000D10700000C
:1000D000DB070000E5070000EF070000F90700005C
:1000E000030800000D0800001708000021080000A8
:1000F0002B080000350800003F08000049080000F8
:10010000530800001FB500F003F88DE80F001FBD75
:1001100000F038BC70B50B46010B184400F6FF70B8
:10012000040B4FF080500022090303692403406947
:1001300043431D1B104600F0E9F929462046BDE85F
:10014000704000F0E3B9F0B54FF6FF734FF4B475AB
:100150001A466E1E12E0A94201D3344600E00C4656
:10016000B1EB040130F8027B641E3B441A44F9D120
:100170009CB204EB134394B204EB12420029EAD17F
:1001800098B200EB134002EB124140EA0140F0BD8F
:10019000C34992B00446D1E90001CDE91001FF2224
:1001A0004021684600F094FB94E80F008DE80F00B2
:1001B000684610A902E004C841F8042D8842FAD12B
:1001C00010216846FFF7BFFF1090AA208DF8440069
:1001D00000F0FAF800F0DDF84FF01024A0691022CA
:1001E0006946803000F0DEF8A069082210A900F00E
:1001F000D9F800F0C2F870B504460068A94D072888
:1002000069D2DFE800F033041929561E2500D4E92D
:10021000026564682946304600F0FDF82A4621460A
:10022000304600F0BFF8AA002146304600F024FB1B
:10023000002800D0032070BD00F0D6FB4FF48050A2
:1002400007E0201D00F0C6F80028F4D100F0CCFB38
:1002500060682860002070BD241D94E807009200AB
:1002600000F00AFB0028F6D00E2070BD00F0BEF8AA
:100270000028FAD1D4E9010100EB81034FF080504E
:10028000026945696A43934209D84FF010225369C5
:1002900003EB81030169406941438B4201D9092085
:1002A00070BD5069401C01D10F2070BD2046FFF782
:1002B0006FFF00F09BF80028F7D1201D00F08AF8AE
:1002C0000028F2D160680028F0D100F07DF800F03D
:1002D00060F800F052F8072070BD10B50C461828E1
:1002E00002D00120086010BD2068FFF784FF206065
:1002F00010BD4FF01024A069401C05D0A569A66967
:1003000080353079AA2808D06069401C2DD06069FA
:100310000068401C29D060692CE010212846FFF7B6
:1003200012FF316881421CD1A16901F18002C03104
:1003300005E030B108CA51F8040D984201D10120FE
:1003400000E000208A42F4D158B1286810B1042896
:1003500003D0FEE7284600F070F85249686808604C
:1003600008E000F016F800F008F84FF4805001683B
:10037000491C01D000F012FBFEE7BFF34F8F4A4843
:1003800001684A4A01F4E06111430160BFF34F8FF5
:10039000FEE74FF010208169491C02D0806900F00F
:1003A0008CB870472DE9F04117460D4606460024EB
:1003B00006E03046296800F093F8641C2D1D361DB8
:1003C000BC42F6D3BDE8F0814FF0102080694FF4B5
:1003D00080519FE64FF080510A69496900684A439D
:1003E000824201D810207047002070474FF08050A3
:1003F0000169406941434FF01020826902F5805243
:10040000914201D2092070478069401C01D0002030
:1004100070470420704770B50C4605464FF480665F
:1004200008E0284600F049F8B44205D3A4F58064FA
:1004300005F58055002CF4D170BD4168044609B122
:10044000012600E000264FF010256869A26892009E
:1004500000F012FAF8B1A06881006869FFF75AFE4F
:10046000BEB16E694FF08050A56864680169426949
:100470005143A1420DD9016940694143A94208D9BC
:1004800029463046FFF7C7FF2A4621463046FFF788
:1004900089FFFFF772FFFFF797FFFFF77AFFF8E793
:1004A0000C0A0000000000200CED00E00400FA053A
:1004B000144801680029FCD07047134A02211160DA
:1004C00010490B68002BFCD00F4B1B1D18600868EF
:1004D0000028FCD00020106008680028FCD070477D
:1004E000094B10B501221A60064A1468002CFCD092
:1004F000016010680028FCD00020186010680028F7
:10050000FCD010BD00E4014004E5014070B50C468C
:10051000054600F073F810B900F07EF828B12146C6
:100520002846BDE8704000F007B821462846BDE8DF
:10053000704000F037B800007FB5002200920192B1
:10054000029203920A0B000B6946012302440AE05F
:10055000440900F01F0651F8245003FA06F635430B
:1005600041F82450401C8242F2D80D490868009A94
:1005700010430860081D0168019A1143016000F0F2
:100580003DF800280AD0064910310868029A104345
:100590000860091D0868039A104308607FBD0000C9
:1005A0000006004030B50F4C002200BF04EB0213E0
:1005B000D3F800582DB9D3F8045815B9D3F8085812
:1005C0001DB1521C082AF1D330BD082AFCD204EB1D
:1005D0000212C2F80008C3F804180220C3F8080881
:1005E00030BD000000E001404FF08050D0F83001F5
:1005F000082801D000207047012070474FF080503C
:10060000D0F83011062905D0D0F83001401C01D0B7
:1006100000207047012070474FF08050D0F8300123
:100620000A2801D0002070470120704708208F4918
:1006300009680958084710208C4909680958084773
:1006400014208A4909680958084718208749096809
:100650000958084730208549096809580847382053
:1006600082490968095808473C20804909680958A7
:10067000084740207D4909680958084744207B49BC
:1006800009680958084748207849096809580847FF
:100690004C20764909680958084750207349096871
:1006A00009580847542071490968095808475820D3
:1006B0006E490968095808475C206C49096809585F
:1006C0000847602069490968095808476420674954
:1006D00009680958084768206449096809580847A3
:1006E0006C20624909680958084770205F49096809
:1006F0000958084774205D49096809580847782057
:100700005A490968095808477C2058490968095816
:1007100008478020554909680958084784205349EB
:100720000968095808478820504909680958084746
:100730008C204E4909680958084790204B490968A0
:1007400009580847942049490968095808479820DA
:1007500046490968095808479C20444909680958CE
:100760000847A0204149096809580847A4203F4983
:10077000096809580847A8203C49096809580847EA
:10078000AC203A49096809580847B0203749096838
:1007900009580847B4203549096809580847B8205E
:1007A0003249096809580847BC2030490968095886
:1007B0000847C0202D49096809580847C4202B491B
:1007C000096809580847C82028490968095808478E
:1007D000CC202649096809580847D02023490968D0
:1007E00009580847D4202149096809580847D820E2
:1007F0001E49096809580847DC201C49096809583E
:100800000847E0201949096809580847E4201749B2
:10081000096809580847E820144909680958084731
:10082000EC201249096809580847F0200F49096867
:1008300009580847F4200D49096809580847F82065
:100840000A49096809580847FC20084909680958F5
:1008500008475FF480700549096809580847000097
:1008600003480449024A034B70470000000000207F
:10087000180A0000180A000040EA010310B59B079F
:100880000FD1042A0DD310C808C9121F9C42F8D0FA
:1008900020BA19BA884201D9012010BD4FF0FF30AB
:1008A00010BD1AB1D30703D0521C07E0002010BDC1
:1008B00010F8013B11F8014B1B1B07D110F8013B4D
:1008C00011F8014B1B1B01D1921EF1D1184610BD2E
:1008D00002F0FF0343EA032242EA024200F005B8B5
:1008E0007047704770474FF000020429C0F0128033
:1008F00010F0030C00F01B80CCF1040CBCF1020FD3
:1009000018BF00F8012BA8BF20F8022BA1EB0C01A7
:1009100000F00DB85FEAC17C24BF00F8012B00F89D
:10092000012B48BF00F8012B70474FF0000200B5C3
:10093000134694469646203922BFA0E80C50A0E802
:100940000C50B1F12001BFF4F7AF090728BFA0E8B0
:100950000C5048BF0CC05DF804EB890028BF40F87C
:10096000042B08BF704748BF20F8022B11F0804FBE
:1009700018BF00F8012B7047014B1B68DB68184754
:100980000000002009480A497047FFF7FBFFFFF706
:10099000B9FB00BD20BFFDE7064B1847064A1060B3
:1009A000016881F30888406800470000180A0000C9
:1009B000180A0000F3020000000000201EF0040FDF
:1009C0000CBFEFF30881EFF30981886902380078E2
:1009D000182803D100E00000074A1047074A1268B0
:1009E0002C3212681047000000B5054B1B68054A01
:1009F0009B58984700BD0000DB020000000000206B
:100A0000080A0000040000000010000000000000C0
:080A100000FFFFFF0090D0037E
:1010000010080020151200001D1200001F12000021
:101010002112000023120000251200000000000031
:101020000000000000000000000000002712000087
:1010300029120000000000002B1200002D120000F9
:101040002F1200002F1200002F1200002F1200009C
:101050002F120000000000002F1200002F120000CD
:101060002F1200002F1200002F1200002F1200007C
:101070002F1200002F1200002F1200002F1200006C
:101080002F1200002F1200002F1200002F1200005C
:101090002F1200002F1200002F1200002F1200004C
:1010A0002F1200002F1200000000000000000000BE
:1010B0002F1200002F1200000000000000000000AE
:1010C0000000000000000000000000000000000020
:1010D0000000000000000000000000000000000010
:1010E0000000000000000000000000000000000000
:1010F00000000000000000000000000000000000F0
:1011000000000000000000000000000000000000DF
:1011100000000000000000000000000000000000CF
:1011200000000000000000000000000000000000BF
:1011300000000000000000000000000000000000AF
:10114000000000000000000000000000000000009F
:10115000000000000000000000000000000000008F
:10116000000000000000000000000000000000007F
:10117000000000000000000000000000000000006F
:10118000000000000000000000000000000000005F
:10119000000000000000000000000000000000004F
:1011A000000000000000000000000000000000003F
:1011B000000000000000000000000000000000002F
:1011C000000000000000000000000000000000001F
:1011D000000000000000000000000000000000000F
:1011E00000000000000000000000000000000000FF
:1011F00000000000000000000000000000000000EF
:10120000DFF80CD000F018F8004800470516000081
:10121000100800200648804706480047FEE7FEE722
:10122000FEE7FEE7FEE7FEE7FEE7FEE7FEE7FEE796
:101230005D12000001120000064C074D06E0E06858
:1012400040F0010394E8070098471034AC42F6D30D
:10125000FFF7DAFF7C1600009C160000F0B5A848E6
:10126000A74B012600781B1D1A1D4FF08051062840
:101270000BD11C78240708D11478C4F30314032C71
:1012800006D0042C04D0052C02D0062807D011E08B
:10129000B1F824439B4DC4F304242C6002E01C7875
:1012A000240707D11478C4F30314032C02D1974DFB
:1012B000954C6C67D1F83051D1F84442944FC4F347
:1012C00042343C6006280CD11C78240709D11478DC
:1012D000C4F30314032C04D18E4C276827F08077C5
:1012E00027604FF080470024C7F80C41C7F8104131
:1012F000874F3F1F3C60062807D11F783F0704D166
:101300001778C7F30317032F02D0062808D01FE071
:10131000DFF8FCC103270CF1640CCCF8007007E087
:101320001F783F0714D11778C7F30317032F0FD186
:10133000DFF8E4C10527CCF80070774F78373E60BE
:10134000754F08373C600CF1040C3F27CCF8007057
:10135000724F3F68DFF8C8C1CCF800706F4F3F1D77
:101360003F680CF1040CCCF800706C4F08373F68F4
:101370000CF1040CCCF80070684F0C373F680CF18E
:10138000040CCCF80070654F10373F680CF1040C6A
:10139000CCF80070614F14373F680CF1040CCCF8A6
:1013A00000705E4F18373F68DFF874C10CF1200CF5
:1013B000CCF80070594F1C373F680CF1040CCCF886
:1013C0000070564F20373F680CF1040CCCF80070C9
:1013D000524F24373F680CF1040CCCF800704F4F8B
:1013E00028373F680CF1040CCCF800704B4F2C37B9
:1013F0003F680CF1040CCCF80070484F30373F6860
:10140000DFF81CC10CF1400CCCF80070434F3437AE
:101410003F680CF1040CCCF80070404F38373F683F
:101420000CF1040CCCF800703C4F3C373F680CF1D9
:10143000040CCCF80070394F40373F680CF1040CB5
:10144000CCF80070DFF8DCC0FB27CCF80070062871
:1014500013D11F783F0710D11778C7F30317032F55
:1014600003D0042F01D0052F07D1D1F85872DFF82F
:10147000B8C007F04F07CCF800702C480268D207BC
:1014800002D06FF001020260062D08D1D1F83401BC
:10149000062804D12648016841F4806101604FF0BC
:1014A0001021D1F80002002803DBD1F80402002843
:1014B00022DA204A166020480368002BFCD015234E
:1014C000C1F800320568002DFCD0C1F80432016873
:1014D0000029FCD0146001680029FCD0BFF34F8FB5
:1014E0000C48F0380168154A01F4E06111430160CD
:1014F000BFF34F8F00BFFDE7124911480860F0BDF0
:10150000E00F00F0403501400DF0ADBA00C00740DB
:101510003C050040FCED00E01056004004040010C3
:1015200020C5004018F50040E40E004000040040D3
:101530003C17004004E5014000E401400400FA05C6
:101540000090D0030800002002E008C8121F08C164
:10155000002AFAD170477047002001E001C1121F34
:10156000002AFBD1704700002DE9FC410646C00768
:101570004FF000050ED0104F00240122385D009579
:1015800000231146019500F055F8641C042CF4D397
:1015900000F02EF8B0070DD5074E0024361D0022AE
:1015A000305D032300951146019500F043F8641C5B
:1015B000042CF4D3BDE8FC817416000007490B5CD1
:1015C0004FF0A041D1F804250120984020EA020301
:1015D000C1F808351040C1F80C05704774160000BA
:1015E0000249085C012100F037B8000074160000C1
:1015F00010B500242046FFF7F3FF641C042CF9D338
:1016000010BD00000120FFF7AFFF094C4FF4FA783E
:101610004FF47A4700263046FFF7D0FF4546611C5D
:10162000384688476D1EFAD1761C042EF3DBF1E7AD
:101630006E16000070B541EA4201DDE904564FF034
:10164000A04441EA830141EA052104EB800041EA1C
:101650000641C0F8001770BD01224FF0A043824040
:1016600011B1C3F808257047C3F80C257047073837
:10167000FDD87047111213140D0E0F109C160000A8
:10168000080000200400000048150000A01600001B
:101690000C00002004080000581500000090D00342
:00000001FF
